TagPDF.com

ocr sdk c#: Mar 6, 2019 · We are sunsetting the MSDN Code Gallery.​ ... .NET Barcode Scanner Library API for .NET Barcode Reading ...



ocr class c# Dynamsoft OCR SDK for .NET













android ocr app handwriting, aquaforest ocr sdk for .net, pdf ocr windows, ocr asp.net sample, ocr software free trial, java pdf ocr api, microsoft ocr library for windows runtime vb.net, js ocr number, azure computer vision api ocr, microsoft azure ocr python, swiftocr cocoapods, c++ ocr, ocr sdk freeware, c# free ocr api, sharepoint ocr pdf search



simple ocr c#


Jun 21, 2018 · IronOCR is an advanced OCR (Optical Character Recognition) & Barcode library for C# and VB.Net. The engine adds OCR functionality to ...

tesseract ocr c# tesseractengine

Cognitive Services – Optical Character Recognition ... - C# Corner
Cognitive Services – Optical Character Recognition ( OCR ) From An Image Using Computer Vision API And C# . Rajeesh Menoth; Jul 13 2018. 10.2k; 0; 5.

In 9, P roviding Services with Interfaces, you created a SortablePoint class that provided a sorting mechanism based on the distance from the origin. With the addition of a shared or static field and property, you can easily sort the points based on the distance from any point. Creating the SortablePoint Class The SortablePoint class will start with X and Y properties, a constructor, and an overridden ToString method as instance members, similar to the implementation in 9. You ll then add a shared or static member Center and modify the CompareTo function to use Center instead of the origin. Finally, you ll implement a shared or static Parse method that s able to read the same string format that the ToString method creates. Create the class 1. Create a new Windows application project. Name it SortablePoint. 2. Add a new class to the project. Name it SortablePoint. 3. Modify the class to indicate that it will implement the IComparable interface. 4. 5. 6. 7. 8. 9. 10. // Visual C# public class SortablePoint : IComparable { Visual Basic Public Class SortablePoint Implements IComparable End Class



c# ocr library


Dec 16, 2018 · Tesseract is probably the most accurate open source OCR engine available. Combined with the Leptonica Image Processing Library it can ...

abbyy ocr sdk c#


Tesseract is a library for reading straight and perfect text of standardized typefaces. To use Tesseract when we are ...

ASP.NET controls are like HTML factories that accept external parameters and produce chunks of markup. As a developer, you can select and filter any parameters being assigned to control properties. As a developer, though, you can hardly control what the component does to generate the markup. The bad effect is that you end up with an HTML markup that might work differently on different browsers and different browser configurations. When this happens, though, the worst thing is that you have no way to fix it the HTML is out of your reach. Before ASP.NET 4, adaptive rendering was the common way to address this problem. Adaptive rendering is the process that enables controls to generate different markup for individual browsers. This result is obtained by delegating the generation of the markup to an external component the adapter. When each control is about to render, it figures out its current adapter and hands the request over to that adapter. Nicely enough, a control adapter is a configurable component that you can declaratively unplug in any application to roll your own. The selected adapter depends on the current browser. The adapter for a control is resolved by looking at the browser capabilities as configured in the ASP.NET browser database. If the browser record includes an adapter class for a given control, the class is instantiated and used. Otherwise, the default adapter for the control is used, which is an instance of the ControlAdapter class. The ControlAdapter class is a generic adapter and simply generates the markup for a control by calling the rendering methods on the control itself. Note The ASP.NET database used for storing browser information is not a real database. It is,





c# microsoft.windows.ocr

Windows -universal-samples/Samples/ OCR at master · microsoft ...
OCR sample . Shows how to use Windows .Media. Ocr API. Optical character ... for this specific sample , then the subfolder for your preferred language (C++, C# , ...

microsoft.windows.ocr c# example


C# ASP.NET VB.NET Optical character recognition OCR API to find and extract text ... Download Free Trial ... NET is a robust optical character recognition API.

Slot 22, Offset 0x165, Length 91, DumpStyle BYTE Record Type = PRIMARY_RECORD Record Size = 91 Memory Dump @0x6292C165 00000000: 00000010: 00000020: 00000030: 00000040: 00000050: 30001800 38303120 3832362d 30373532 0...801 826-0752 55543834 313532ff 09000000 05003300 UT84152 .....3. 39003f00 4d005b00 3939382d 37322d33 9. .M.[.998-72-3 35363752 696e6765 72416c62 65727436 567RingerAlbert6 37205365 76656e74 68204176 2e53616c 7 Seventh Av.Sal 74204c61 6b652043 697479 t Lake City Record Attributes = NULL_BITMAP VARIABLE_COLUMNS

18

In the following exercise, you will use the SaveFileDialog class. In the BellRingers application, when the user saves details to a le, you will prompt the user for the name and location of the le by displaying the Save File common dialog box.

By default, Word displays the ruler in Normal, Web Layout, and Print Layout views and does not display the ruler in Outline and Reading Layout views. If you don t see the ruler in Nor mal, Web Layout, or Print Layout view, you can display it by choosing View, Ruler.

public class ProductsService : IProductsService { }

tesseract ocr c#

OCR using Tesseract in C# - C# Corner
7 Mar 2016 ... In this article I am going to show how to do OCR using Tesseract in C# .

onenote ocr in c#


Sep 18, 2014 · Windows apps · OneDrive · Outlook · Skype · OneNote ... We are pleased to announce that Microsoft OCR Library for Windows Runtime has ... for example you can recognize patterns such as email addresses, phone numbers, and ... The extracted text and layout info are contained within OcrResult: C# 2.

C# also provides two other loop constructions, called do while and while. These are not really vital in that you can always get the looping behavior that you want by using an appropriately designed for loop, but they can be useful in situations where you don t want to go to the trouble of creating a for loop construction. You can find out more about these kinds of loops and when they would be useful in the glossary.

8

c# ocr nuget


A simple example of testing Tesseract OCR in C#: .... Tesseract OCR 3.02.02 API can be confusing, so this guides you through including the ...

tesseract ocr pdf c#

OCR using Tesseract in C# - C# Corner
7 Mar 2016 ... Next Recommended Article Cognitive Services – Optical Character Recognition ( OCR ) From An Image Using Computer Vision API And C# .












   Copyright 2021.